:020000040000FA
:10000000006AEDEF00F0E950086E849084948494C7
:100010009690969496940F0E9316085000B222D0A4
:100020003A0E026E980EB4EC00F0330E076E2FD825
:10003000130E026E880EB4EC00F029D8640EB3ECF7
:1000400000F025D8640EB3EC00F0220E076E1FD826
:10005000280E07D80C0E05D8060E03D800820850CB
:1000600001D00080076E00A00BD0849403080EE33B
:100070000DD80F0E026EA00EB4EC00F0D880120066
:100080000080FE08D8B4EAEF00F0848400A000905D
:1000900084800F0E81160750F00B8112000000D0F3
:1000A000000000D08490073A000000D0000000D08B
:1000B00000B0EDD7C80EB3EC00F0D880EAEF00F046
:1000C000159E0A50D8B4158E050E096E270E046EC3
:1000D000100E0CD8030E046EE80E08D8046A640EE5
:1000E00005D8046A0A0E02D8055008D0036E0650DF
:1000F000026E0550016ECCEC00F00150016E094E0D
:10010000159E0A5003E0095CD8B012000150D8A433
:10011000159E15BE1200300FE4EF00F0E836E83609
:100120003C0B0109C212C009C216C050F80B0309EA
:10013000C06E000E026E320EB4EC00F0C282C2B28B
:10014000FED7026AC450EAEF00F0046A036EFF0EA5
:100150000326D8A00426D8A0EAEF00F0030E026E12
:10016000E70E02D8F4D7026AFD0F016EFF0E00D031
:1001700001D00126040000D000D0D8A00226D8A0CB
:100180001200F7D7086E0A0E036E046ACCEC00F07A
:100190000806FCE705501200066A056A100E076E95
:1001A0000234053606360350055E0450065A05E251
:1001B0000350052604500622D89001360236072E39
:1001C000EFD70150EAEF00F0E96EFB6A1250FA6EC9
:1001D0001150F96E000104001200D7EF04F0120C68
:1001E000010C100C010C020C000C000C080CD80CBB
:1001F000040C0A0C000C000C000C010C020C030C8B
:10020000010C06020602090C020C430C000C020C45
:10021000010C020C800C500C090C040C000C000C9E
:10022000010C020C020C010C000C050C240C000C3F
:10023000100C010C040C240C020C020C050C240CF8
:10024000060C000C010C050C240C010C000C010C1C
:10025000070C050C820C030C080C000C020C090C9A
:10026000040C010C000C020C0A0C000C000C000C1D
:10027000070C050C030C020C400C000C000C070CC6
:10028000050C830C020C400C000C000C96029E0224
:10029000C602FE021A03040C030C090C040C140C15
:1002A000030C4D0C000C690C000C630C000C720C60
:1002B000000C6F0C000C630C000C680C000C690C3B
:1002C000000C700C000C1C0C030C500C000C490CA6
:1002D000000C430C000C310C000C380C000C200CF2
:1002E000000C550C000C530C000C420C000C200CA4
:1002F000000C430C000C440C000C430C000C0E0CC6
:10030000030C560C000C310C000C2E0C000C310CA4
:10031000000C460C000C530C000C0A0C030C430C94
:10032000000C660C000C670C000C310C000C040176
:100330002E51600B00083EE1050E2F6303D0040E22
:100340002A6F36D0060E2F6301D035D0080E2F63EA
:1003500009D02B0E226F040E236F010E286F296B1C
:100360002D9326D0090E2F6301D06AD0000E2F6383
:1003700001D07ED0010E2F6301D09FD0030E2F63DA
:1003800001D09BD00A0E2F630BD02C0E226F040ECF
:10039000236F32512227010E286F296B2D9308D02D
:1003A0000B0E2F63120024EE2CF0325130C4DBFF11
:1003B000010E276F1200800E2E631200010E3163B2
:1003C0000FD0DE0E226F010E236F22C4F6FF23C46E
:1003D000F7FFF86A0800F5CF28F4296B2D83E8D7DA
:1003E000020E316312D0060E226F020E236F0A0E28
:1003F000F66E020EF76EF86A0900F5CF28F40900D0
:100400000900F5CF29F42D83D3D7030E31631200F1
:10041000F86AF76A30458C0FF66E020EF722090073
:10042000F5CF22F40800F5CF23F422C4F6FF23C44D
:10043000F7FFF86A0800F5CF28F4296B2D83B8D7A9
:10044000010E276F2FEE71F00F0EDE6AE82EFDD73A
:1004500024EE2CF0010EDE6AE82EFDD730512B6F12
:1004600003E1050E2A6F1200060E2A6F08DA120049
:10047000366B376B2E511F0B000803E12DB136830D
:100480000ED02E511F0B010801E109D02E511F0B78
:10049000020807E134D8DF50040B01E03681010E79
:1004A000276F010E27631200360E226F040E236F92
:1004B000020E286F296B2D931200010E306309D0B4
:1004C0002E511F0B000805E12D81030E2F632D9186
:1004D0006FD7000E306312002E511F0B0208FBE194
:1004E00032510F0BF8E00BD8030E2F6303D0840EAC
:1004F000DF6E5ED7000E32AF880EDF6E59D724EE66
:1005000000F032453235E846E846D9261200000EA2
:100510006C6205D000513C0B340805E010D0040E8D
:100520006C62120015D0000E266F000E276F286B2C
:10053000296BFDDE000E276379D045D977D0020EF6
:100540002663AFD057D8C80E00BD880E006F1200CA
:10055000040E2A6306D030516E6E050ED8B4030E19
:100560002A6F010E26639DD005D8C80E04BD880EE3
:10057000046F12002851206F2951216F000804E3F5
:1005800007E12851080804E2080E206F000E216FD1
:100590002051056F285F2151295B0451FC0B21116B
:1005A000046F24EE36F0215102E1205122E02DA308
:1005B00012D022C4F6FF23C4F7FFF86A0900F5CF72
:1005C000DEFF09002007FAE12107F8E2F6CF22F466
:1005D000F7CF23F4120022C4E1FF23C4E2FFE6CFE9
:1005E000DEFF2007FCE12107FAE2E1CF22F4E2CFAF
:1005F00023F412000151206F28270051030B216FB3
:10060000292314EE36F024C4D9FF25C4DAFF215182
:1006100002E120510AE0E6CFDEFF2007FCE12107DE
:10062000FAE2D9CF24F4DACF25F41200000E2763C2
:100630000AD0080E016F2E0E026F040E036F840E97
:10064000006F046F2CD02EAF1DD02951355D04E30F
:1006500007E12851345D04E234C428F435C429F498
:1006600089DF010E266F080E016F2E0E026F040E39
:10067000036F800E006F360E066F040E076FC80EF4
:10068000046F0DD0020E266F056BC80E046F080EA6
:10069000016F360E026F040E036FC80E006F6D9867
:1006A0001200000E266F080E016F2E0E026F040E50
:1006B000036F880E006F000E046F12000401140E09
:1006C0006F6E000E2A6F2D6B2B6BD9D812000401B0
:1006D0006DA60CD8010E2A6312006DBA1200686A6A
:1006E000696A69806988020E2A6F12006D6A696AF8
:1006F0006D86010E2A6F120004016D6A696A000E90
:100700002A6F12000401000E2A5D23E068A402D0C3
:1007100069B424D86DB2120068A002D069B039D88B
:1007200068A802D069B816D868AC02D069BC28D8CD
:1007300068AA02D069BA26D868A202D069B227D8BE
:10074000030E2A5D06E368A604D069A602D0DFDEA8
:1007500068961200698468986D8212006D9269949F
:100760006894120004012DA11200F8DF6D84100EB0
:10077000DA6ED96AD92EFED7DA2EFCD76D94120024
:10078000689C120070B08DDF7090689A12006892B9
:1007900012006A6A686A9F0E6B6E7B0E696E6E6AE3
:1007A0002FEE71F00F0EDE6AE82EFDD7160E706E7A
:1007B00068B6689668B6FDD76D9873DF2D912B6B80
:1007C000030E2A6F120004012E511F0B010809E1CC
:1007D0002E51600B200805E1000E325D03E0010E92
:1007E00032631200000E2F6309D0460E226F040EF2
:1007F000236F2D93080E286F296B3ED0010E2F63B7
:1008000005D0460E246F040E256F36D0020E2F63DE
:1008100001D01200030E2F6301D01200040E2F63CB
:1008200001D01200200E2F6305D03E0E246F040E5F
:10083000256F22D0210E2F6314D0000E3E6FC20E02
:100840003F6F010E406F416B426B436B080E446F6C
:100850003E0E226F040E236F2D93070E286F296B17
:100860000BD0220E2F6303D030C445F405D0230EE5
:100870002F6301D012001200030E276F1200020E28
:10088000E96E14EE4EF0080E0CD8030EE96E14EE6D
:1008900057F0400E1CD8030EE96E14EE98F0400E8F
:1008A00000D0E66E2FEE70F0E950D9261A0EDF1256
:1008B000E944E846E84604EE04F0E926020EE1CFFA
:1008C000EBFF030EE2CFEBFF400EEF6E1200E66E81
:1008D0002FEE70F0E950D9261C0EDF12E944E846ED
:1008E000E84604EE00F0E926020EE1CFEBFF030E2E
:1008F000E2CFEBFFE550E92AE7CFEDFF880EEF6E80
:100900001200016E0401060E2A5D000ED89009E166
:10091000E944E846E84604EE04F0E926000ED890E3
:10092000EFBE1200020EEBCFD9FF030EEBCFDAFFC2
:10093000FF0EDB500160016EE92A0150ED6E04E00C
:10094000E6CFDEFFE82EFCD7400EEF16EF7C880ED8
:10095000EF120150D8801200016E0401060E2A5DCC
:10096000000ED89009E1E944E846E84604EE00F0BC
:10097000E926000ED890EFBE1200020EEBCFD9FF91
:10098000030EEBCFDAFFEC500160016EFF0EDB507F
:10099000ED6E015004E0DECFE6FFE82EFCD7400EFE
:1009A000EF16EF7C880EEF120150D8801200FF0E78
:1009B000926E0A0EC16E84929692010E046EF40E2F
:1009C000A6EC00F0226AFE0E04EC00F0010E04EC2E
:1009D00000F0550E04EC00F0530E04EC00F0420E53
:1009E00004EC00F0200E04EC00F0520E04EC00F0D9
:1009F000650E04EC00F0610E04EC00F0640E04ECF3
:100A000000F0790E04EC00F059DEEAEC00F0829080
:100A100094905DDE77DEEAEC00F0100E1E6E030EA1
:100A2000E96E10EE26F01E5097DFEAEC00F01E6E25
:100A3000D8A0EFD726C023F08270949004002350F2
:100A40003008D8A487EF05F0206A04000F0E205C60
:100A5000D8B05BEF05F02050F66E0E08D8A050EF2E
:100A600005F0F76AF86AD890F636F736820EF62661
:100A70000A0EF722000EF8220800F5CF1FF050EF03
:100A800005F0480C650C6C0C6C0C6F0C200C570CB2
:100A90006F0C720C6C0C640C210C0D0C0A0C000C0D
:100AA0002050260FE96E000EEA6AEA221FC0EFFF0F
:100AB000202AD8A4CAD7FE0E04EC00F0C00E04EC25
:100AC00000F0480E04EC00F0650E04EC00F06C0E33
:100AD00004EC00F06C0E04EC00F06F0E04EC00F07F
:100AE000200E04EC00F0570E04EC00F06F0E04EC46
:100AF00000F0720E04EC00F06C0E04EC00F0640EDA
:100B000004EC00F0210E04EC00F03CEF08F00400CF
:100B100023503108D8A4FDEF05F0010E8EEC00F053
:100B20001C6E320EA5EC00F0310E1D6EFE0E04ECB4
:100B300000F0C00E04EC00F0200E04EC00F0200EDB
:100B400004EC00F0410E04EC00F0440E04EC00F064
:100B5000430E04EC00F0200E04EC00F0430E04EC15
:100B600000F0680E04EC00F0200E04EC00F0310EF2
:100B700004EC00F0200E04EC00F0200E04EC00F079
:100B8000FE0E04EC00F0940E04EC00F0200E04ECD9
:100B900000F0200E04EC00F0200E04EC00F0200E1B
:100BA00004EC00F0200E04EC00F0200E04EC00F049
:100BB000200E04EC00F0200E04EC00F0200E04ECFB
:100BC00000F0200E04EC00F0200E04EC00F0200EEB
:100BD00004EC00F0FE0E04EC00F0940E04EC00F0C7
:100BE0000A6A1CC005F0066A060E116E126A60ECF5
:100BF00000F04FEC08F03CEF08F0040023503208FE
:100C0000D8A473EF06F0020E8EEC00F01C6E320ECC
:100C1000A5EC00F0320E1D6EFE0E04EC00F0C00ECE
:100C200004EC00F0200E04EC00F0200E04EC00F0C8
:100C3000410E04EC00F0440E04EC00F0430E04EC12
:100C400000F0200E04EC00F0430E04EC00F0680EFF
:100C500004EC00F0200E04EC00F0320E04EC00F086
:100C6000200E04EC00F0200E04EC00F0FE0E04EC6C
:100C700000F0940E04EC00F0200E04EC00F0200EC6
:100C800004EC00F0200E04EC00F0200E04EC00F068
:100C9000200E04EC00F0200E04EC00F0200E04EC1A
:100CA00000F0200E04EC00F0200E04EC00F0200E0A
:100CB00004EC00F0200E04EC00F0200E04EC00F038
:100CC000FE0E04EC00F0940E04EC00F00A6A1CC066
:100CD00005F0066A060E116E126A60EC00F04FEC29
:100CE00008F03CEF08F0040023503308D8A4E9EFE3
:100CF00006F0030E8EEC00F01C6E320EA5EC00F038
:100D0000330E1D6EFE0E04EC00F0C00E04EC00F07D
:100D1000200E04EC00F0200E04EC00F0410E04EC78
:100D200000F0440E04EC00F0430E04EC00F0200E42
:100D300004EC00F0430E04EC00F0680E04EC00F04C
:100D4000200E04EC00F0330E04EC00F0200E04EC56
:100D500000F0200E04EC00F0FE0E04EC00F0940E07
:100D600004EC00F0200E04EC00F0200E04EC00F087
:100D7000200E04EC00F0200E04EC00F0200E04EC39
:100D800000F0200E04EC00F0200E04EC00F0200E29
:100D900004EC00F0200E04EC00F0200E04EC00F057
:100DA000200E04EC00F0200E04EC00F0FE0E04EC2B
:100DB00000F0940E04EC00F00A6A1CC005F0066A0C
:100DC000060E116E126A60EC00F04FEC08F03CEF7A
:100DD00008F0040023503408D8A45FEF07F0040E95
:100DE0008EEC00F01C6E320EA5EC00F0340E1D6E81
:100DF000FE0E04EC00F0C00E04EC00F0200E04EC3B
:100E000000F0200E04EC00F0410E04EC00F0440E63
:100E100004EC00F0430E04EC00F0200E04EC00F0B3
:100E2000430E04EC00F0680E04EC00F0200E04EC1D
:100E300000F0340E04EC00F0200E04EC00F0200E64
:100E400004EC00F0FE0E04EC00F0940E04EC00F054
:100E5000200E04EC00F0200E04EC00F0200E04EC58
:100E600000F0200E04EC00F0200E04EC00F0200E48
:100E700004EC00F0200E04EC00F0200E04EC00F076
:100E8000200E04EC00F0200E04EC00F0200E04EC28
:100E900000F0200E04EC00F0FE0E04EC00F0940EC6
:100EA00004EC00F00A6A1CC005F0066A060E116E1A
:100EB000126A60EC00F04FEC08F03CEF08F0040020
:100EC00023503508D8A408EF08F0222AFE0E04ECBF
:100ED00000F0D40E04EC00F0200E04EC00F0200E24
:100EE00004EC00F0200E04EC00F0200E04EC00F006
:100EF000200E04EC00F0200E04EC00F0200E04ECB8
:100F000000F0200E04EC00F0200E04EC00F0200EA7
:100F100004EC00F0200E04EC00F0200E04EC00F0D5
:100F2000FE0E04EC00F0D40E04EC00F0560E04ECBF
:100F300000F0610E04EC00F06C0E04EC00F0750E95
:100F400004EC00F0650E04EC00F03D0E04EC00F043
:100F50000A6A22C005F0066A060E116E126A60EC7B
:100F600000F0206A0400070E205CD8B0E0EF07F024
:100F70002050F66E0608D8A0D5EF07F0F76AF86A99
:100F8000D890F636F7369C0EF6260F0EF722000E96
:100F9000F8220800F5CF1FF0D5EF07F0560C610CD2
:100FA0006C0C750C650C200C3D0C2050260FE96E66
:100FB000000EEA6AEA221FC0EFFF202AD8A4D2D787
:100FC00022C001F0026A020EC2EC00F0136E146A35
:100FD000300E13242D6E22C001F0026A010EC2EC05
:100FE00000F0136E146A300E13242E6E22C001F02E
:100FF000026A000EC2EC00F0136E146A300E132465
:101000002F6E0D0E306E0A0E316E326A3CEF08F014
:10101000206A04000E0E205CD8B03CEF08F020508F
:10102000F66E0B08D8A031EF08F0F76AF86AD8908E
:10103000F636F7364A0EF626100EF722000EF82284
:101040000800F5CF1FF031EF08F0450C6E0C740C62
:10105000650C720C200C300C2D0C350C0D0C0A0C90
:10106000000C2050260FE96E000EEA6AEA221FC02B
:10107000EFFF202AD8A4CDD767EC03F082EC03F071
:10108000EAEC00F0030EE96E10EE26F00F0E81EC94
:1010900004F0EAEC00F0D8A0EFD709EF05F0410E1C
:1010A000266E640E276E630E286E1DC029F03D0E5D
:1010B0002A6E1CC001F0026A020EC2EC00F0136E30
:1010C000146A300E13242B6E1CC001F0026A010E4C
:1010D000C2EC00F0136E146A300E13242C6E1CC088
:1010E00001F0026A000EC2EC00F0136E146A300EBA
:1010F00013242D6E0D0E2E6E0A0E2F6E306A120006
:020000040030CA
:08000000E4FEFFF3FFFD9BFF8E
:00000001FF
